:100000000C9490050C94D8050C94D8050C94D80544
:100010000C94D8050C94D8050C94D8050C94D805EC
:100020000C94D8050C94D8050C94E1130C94B314DB
:100030000C9454220C94D8050C94D8050C94D80533
:100040000C94D8050C94D8050C94D8050C94D805BC
:100050000C94D8050C94C8220C94D8050C94D8059F
:100060000C94D8050C94D8050C94D8050C94D8059C
:100070000C94D8050C94D8050C94D8050C94D8058C
:100080000C94D8050C94D8050C94D8050C94D8057C
:100090000C94D8050C94D8050C94D8050C94D8056C
:1000A0000C94D8050C94D8050C94D8052F12561230
:1000B0004E1356124E13A212C5124E131C132B13BD
:1000C00084188418AE18AE1809193D194B1B4B1B28
:1000D00054194B1B3F1A3F1A051B4B1B1A1B381B8D
:1000E000041607090B0A1D1B06196405141A0815C6
:1000F0001C171E1F202123222E26242D25273012D7
:10010000182F0C13280F0D340E33313638111037D9
:100110002B2C352A5829787B79397A504F515272D5
:100120006C63685680668053020103555880576D92
:100130006E5462595A5B5C5D5E5F6F606174756698
:100140003E3F403C4142774476466B47804365459D
:100150008048494A4B4C3D4D3B4E3A7D7E7C7F73F7
:100160000A0025303458006164625F686F73745F01
:100170006B62645F726563763A20004552524F525B
:100180003A206D65646961206B6579300A004552DB
:10019000524F523A206D65646961206B6579310A6E
:1001A000004D3A64657465637420616761696E0A25
:1001B00000544D353A206578740A00556E6B6E6FA9
:1001C000776E0A00544D353A2064656661756C742B
:1001D0000A005D206370693D25640A0025303258AD
:1001E00020004578743A205B00436C617373696347
:1001F000203230306370690A00436C617373696345
:10020000203130306370690A004D3A6164647225B0
:100210006420726567333A20253034580A004D3A1D
:100220006D6F7665206661696C0A004D3A616464A1
:1002300072256420726567333A20253034580A00ED
:100240004D3A5B423A2530325820583A25642825E9
:10025000642920593A25642825642920413A2564D7
:100260005D0A004D3A5B2530325820253032582047
:1002700025303258202530325820253032585D0A3A
:100280000020616464723A25642C20726567333AF9
:10029000253034580A000A5363616E3A0A004D65EE
:1002A000646961206B6579730A0068616E646C65CE
:1002B000723A20253032582C2049534F3A2025736A
:1002C0000A000A4B6579626F6172643A0A00730032
:1002D000530052000A4B6579626F61726420737437
:1002E0006172742E0A000A55534220636F6E66696C
:1002F00067757265642E0A000A0A544D4B3A6365AD
:100300003565353635662B2F4C5546410A0A002E89
:100310000341004400420020006B00650079006248
:10032000006F00610072006400200063006F006EC7
:100330000076006500720074006500720000000E17
:100340000374002E006D002E006B002E00000004D0
:1003500003090409027400040100A032090400002A
:1003600001030101000921110100012240000705DC
:10037000810308000A0904010001030102000921A8
:1003800011010001224D000705820308000A09043B
:1003900002000103000000092111010001223600C2
:1003A0000705830308000A09040300020300000094
:1003B0000921110100012222000705840320000108
:1003C000070504032000011201100100000008EDE0
:1003D000FEDB0A0101010200010631FF0974A101DF
:1003E0000975150026FF009520750881020976150C
:1003F0000026FF00952075089102C005010980A123
:100400000185021601002637001A81002AB70075FF
:100410001095018100C0050C0901A1018503160199
:1004200000269C021A01002A9C0275109501810089
:10043000C005010902A1010901A10005091901294D
:10044000051500250195057501810295017503814A
:10045000010501093009311581257F950275088153
:100460000609381581257F950175088106050C0A56
:1004700038021581257F950175088106C0C00501E8
:100480000906A101050719E029E7150025019508CE
:100490007501810295017508810105081901290579
:1004A00095057501910295017503910105071900E4
:1004B00029FF150026FF00950675088100C0636FAF
:1004C0006E73756D65723A20253034580A00737961
:1004D0007374656D3A20253034580A000A002530BF
:1004E000325820006B6579626F6172643A20004C6B
:1004F00045443A20253032580A00253032583A20F7
:100500002530386225730A00722F63203031323370
:10051000343536370A00290A002575002F00257565
:10052000005D28002564002000256400200025646B
:100530000020002564007C0025303258006D6F7566
:1005400073656B6579205B62746E7C7820792076A8
:1005500020685D287265702F61636C293A205B000A
:100560006D6B5F776865656C5F74696D655F746FEF
:100570005F6D6178203D2025640A006D6B5F7768B0
:1005800065656C5F6D61785F7370656564203D20A3
:1005900025640A006D6B5F74696D655F746F5F6DD4
:1005A0006178203D2025640A006D6B5F6D61785F86
:1005B0007370656564203D2025640A006D6B5F697A
:1005C0006E74657276616C203D2025640A006D6B47
:1005D0005F64656C6179203D2025640A006D6B5F66
:1005E000776865656C5F74696D655F746F5F6D6179
:1005F00078203D2025640A006D6B5F776865656C27
:100600005F6D61785F7370656564203D2025640AC5
:10061000006D6B5F74696D655F746F5F6D617820ED
:100620003D2025640A006D6B5F6D61785F737065B6
:100630006564203D2025640A006D6B5F696E7465FA
:100640007276616C203D2025640A006D6B5F6465E5
:100650006C6179203D2025640A000A00257500366A
:100660003A20776865656C5F74696D655F746F5F6C
:100670006D61783A20000A00257500353A207768C8
:1006800065656C5F6D61785F73706565643A2000C5
:100690000A00257500343A2074696D655F746F5FD8
:1006A0006D61783A20000A00257500333A206D61AB
:1006B000785F73706565643A20000A002575003222
:1006C0003A20696E74657276616C286D73293A20E0
:1006D000000A00257500313A2064656C6179282A8A
:1006E00031306D73293A20000A092D2056616C754E
:1006F0006573202D0A004D3E004D25643E20003FCD
:10070000007365742064656661756C740A00433E0D
:10071000200077686572652064656C74613A2063B7
:100720007572736F723D25642C20776865656C3D2A
:1007300025640A53656520687474703A2F2F656EBE
:100740002E77696B6970656469612E6F72672F77A8
:10075000696B692F4D6F7573655F6B6579730A00FF
:100760000A092D204D6F7573656B6579202D0A453B
:1007700053432F713A09717569740A313A096465F6
:100780006C6179282A31306D73290A323A09696E11
:1007900074657276616C286D73290A333A096D614C
:1007A000785F73706565640A343A0974696D655FD2
:1007B000746F5F6D61780A353A09776865656C5FBB
:1007C0006D61785F73706565640A363A09776865AC
:1007D000656C5F74696D655F746F5F6D61780A0A3F
:1007E000703A097072696E742076616C7565730A6F
:1007F000643A097365742064656661756C74730A84
:1008000075703A092B310A646F776E3A092D310AF7
:10081000706775703A092B31300A7067646F776EB4
:100820003A092D31300A0A7370656564203D2064F1
:10083000656C7461202A206D61785F7370656564F2
:10084000202A2028726570656174202F2074696DDC
:10085000655F746F5F6D6178290A003F004D3E202F
:1008600000433E20004C25640A000A092D20436FF6
:100870006E736F6C65202D0A4553432F713A0971D1
:100880007569740A6D3A096D6F7573656B65790AE0
:10089000000A092D204D61676963202D0A643A0919
:1008A00064656275670A783A096465627567206DE8
:1008B00061747269780A6B3A096465627567206BC6
:1008C0006579626F6172640A6D3A09646562756781
:1008D000206D6F7573650A763A0976657273696F74
:1008E0006E0A733A097374617475730A633A096323
:1008F0006F6E736F6C65206D6F64650A302D343ACE
:10090000096C61796572302D34284631302D4634BA
:10091000290A506175733A09626F6F746C6F616474
:1009200065720A003F0074696D65725F726561648B
:10093000333228293A202530346C580A006B657907
:10094000626F6172645F69646C653A2025580A00C1
:100950006B6579626F6172645F70726F746F636FE1
:100960006C3A2025580A00686F73745F6B65796272
:100970006F6172645F6C65647328293A2025580A98
:10098000000A092D20537461747573202D0A0047E5
:1009900043433A20352E342E30204156522D4C49B7
:1009A00042433A20322E302E30204156525F41527F
:1009B00043483A20617672350A004F5054494F4EF1
:1009C000533A204C554641204D4F5553454B4559C0
:1009D0002045585452414B455920434F4E534F4C9C
:1009E0004520434F4D4D414E44204B45594D4150BC
:1009F0005F53454354494F4E20343039360A004244
:100A000055494C443A2063653565353635662B20AB
:100A10002830393A30323A3133204665622031335A
:100A20002032303230290A005649443A2030784684
:100A300045454428742E6D2E6B2E29205049443A8A
:100A40002030783041444228414442206B6579622D
:100A50006F61726420636F6E7665727465722920AF
:100A60005645523A203078303130310A00444553EF
:100A7000433A20636F6E7665727420414442206B66
:100A80006579626F61726420746F205553420A0069
:100A90000A092D2056657273696F6E202D0A000AAF
:100AA0006D6F7573653A206F66660A000A6D6F7523
:100AB00073653A206F6E0A000A6B6579626F617226
:100AC000643A206F66660A000A6B6579626F61722C
:100AD000643A206F6E0A000A6D61747269783A2078
:100AE0006F66660A000A6D61747269783A206F6EEB
:100AF0000A000A64656275673A206F6E0A000A642C
:100B0000656275673A206F66660A000A0A626F6F4F
:100B1000746C6F616465722E2E2E2000433E20009F
:100B200011241FBECFEFDAE0DEBFCDBF04B603FE57
:100B300028C08091800390918103A0918203B0919D
:100B400083038730904BA740B04BD9F410928003B9
:100B500010928103109282031092830314BE0FB689
:100B6000F894A8958091600088618093600010924D
:100B700060000FBE1092010810920008E0E0F8E358
:100B8000099511E0A0E0B1E0E4E4F6E502C00590CB
:100B90000D92A235B107D9F723E0A2E5B1E001C07B
:100BA0001D92A038B207E1F70E94480F0C94202B49
:100BB0000C940000FF93EF93E0915201F0915301E8
:100BC000309709F00995EF91FF910895FC01859107
:100BD000803011F0EFDFFBCF0895FF27E0E230E235
:100BE00047FF0CC0419597FF09C0EDE260957095F5
:100BF00080959095611D711D811D911D27FF02C07B
:100C0000219530E350E2AA27660F771F881F991FAE
:100C1000AA1FA41710F0A41B63955A95A9F7AA3030
:100C200008F0A95FA05DAF93F3956115710581058B
:100C3000910541F7ED3211F4EF93F395F21718F4A3
:100C40003F93F395FBCF8F91B5DFFA95E1F70895C8
:100C5000E991F9918591803021F0853219F0AADF70
:100C6000F9CF089520E0E89455915532C1F35033FF
:100C700011F4689455915A3348F4505390F3220F6D
:100C8000022E220F220F200D250FF4CF0EF42195F6
:100C900089919991533619F3533729F1533559F105
:100CA000BC0188279927E8945C3621F489919991B1
:100CB00068945591543639F446EF7EF077FF0DC0B5
:100CC0008FEF9FEF0AC055374AE039F0583540E1C1
:100CD00021F0523642E009F00895FF93EF937DDF53
:100CE000EF91FF91B7CFFF93EF93FC01819180309B
:100CF000B9F360DFFBCFFF93EF9368DFF1CFDF93B2
:100D0000CF93CDB7DEB72596A3DFCF91DF910895BE
:100D1000282F2770E82FE695E695E695EF70F0E02E
:100D2000E05AFE4F87FF0AC081E090E001C0880FC3
:100D30002A95EAF780959081892308C081E090E0A8
:100D400001C0880F2A95EAF79081892B8083089546
:100D50000F931F93CF93DF9386E992E09F938F9336
:100D60000E947F060F900F90C0E0D0E001E812E0F3
:100D700063E08C2F0E94F40B009771F09F938F9388
:100D8000DF93CF931F930F930E947F060F900F90D6
:100D90000F900F900F900F902196C031D10541F721
:100DA000DF91CF911F910F9108953F924F925F92E3
:100DB0006F927F928F929F92AF92BF92CF92DF926B
:100DC000EF92FF920F931F93CF93DF93CDB7DEB7D0
:100DD00028970FB6F894DEBF0FBECDBF80915901A2
:100DE00090915A010E949E220C9708F484C20E949E
:100DF000862290935A0180935901809157019091D6
:100E000058010E949E22893E934008F458C10E94D6
:100E100086229093580180935701EBEB4E2EE1E030
:100E20005E2EF4EC6F2EF1E07F2EA2EECA2EA1E032
:100E3000DA2EBCEDAB2EB1E0BB2E63E083E00E9466
:100E4000F40B8C01009709F43AC11F938F931F9202
:100E500083E08F938BE292E09F938F930E947F06B3
:100E600083E00E94650C412F4F602EEF63E083E02A
:100E70000E94530C8FE00E94650C63E08FE00E949B
:100E8000F40B8C010F900F900F900F900F900F901C
:100E9000009729F0982E74E6E72EF12C69C08EE1B8
:100EA00092E09F938F930E947F060F900F90C5CF83
:100EB0008FE00E94650C24E0412F63E08FE00E94E8
:100EC000530C63E08FE00E94F40B8C01982E31E00C
:100ED00083130FC08FE00E94650C22E0412F63E076
:100EE0008FE00E94530C63E08FE00E94F40B8C01B2
:100EF000982E1F930F931F928FE08F9369E072E0FB
:100F00007F936F930E947F060F900F900F900F902A
:100F10000F900F9091E0991230C029EF31E03F938C
:100F20002F930E947F06F0921301E09212010F901E
:100F30000F908FE00E94650C412F407F4A602EEF9A
:100F400063E08FE00E94530C8AE00E94650C63E02E
:100F50008FE00E94F40B8C01982E892B09F46DCF41
:100F600081EA91E09F938F930E947F060F900F90EC
:100F70008FEF890D823088F49BCF62E096120DC00E
:100F800089EE91E09F938F930E947F0668EC70E05A
:100F90007093130160931201CACF74E0971271C06D
:100FA00028E0AE014F5F5F4F61E08FE00E946F0B62
:100FB000863050F02D813E8132272327322730930F
:100FC00013012093120106C0F0921301E092120166
:100FD0008823B9F1882E912C1F928F93DF92CF92A4
:100FE0000E947F060F900F900F900F90312C832D51
:100FF000032C000C990B881599059CF4E1E0F0E0B6
:10100000EC0FFD1FE80FF91F80811F928F93BF9295
:10101000AF920E947F0633940F900F900F900F9025
:10102000E6CF809113018F93809112018F9382ED0F
:1010300091E09F938F930E947F060F900F900F90E7
:101040000F9089818B34C1F48A818D34A9F48B810E
:101050008C3491F48C81813379F47F926F920E9469
:101060007F068FE00E94650C2EEF412F407F63E0EA
:101070008FE00E94530C5BCF5F924F920E947F06DD
:1010800056CF32E3931255CF61EB71E07F936F93AC
:101090000E947F068FE00E94650C28E04AE051E044
:1010A00062E08FE00E941A0C8FE00E94650C28E03D
:1010B00042E051E062E08FE00E941A0C38CF25E058
:1010C000AE014F5F5F4F60E08AE00E946F0B182F08
:1010D000823010F481E00DC18D811F928F938C813D
:1010E0001F928F938B811F928F938A811F928F9370
:1010F00089811F928F9383E692E09F938F930E9442
:101100007F060FB6F894DEBF0FBECDBF123049F494
:10111000998196FB992790F98A8186FB882780F927
:101120000AC0FE01E10FF11D808186FB992790F92D
:1011300082FB882780F948EF58E81530E0F4212F2A
:10114000012E000C330BE1E0F0E0EC0FFD1FE20F8D
:10115000F31F911102C0508301C04083882349F0DE
:10116000E1E0F0E0EC0FFD1FE20FF31F20812760AC
:1011700020831F5FE2CF2D8123FF02C080E001C0EA
:1011800080E827FF80644C8143FF806247FF8061D5
:101190006B8163FF886067FF84603A8137FF8260FC
:1011A000598157FF816080935B01A62FA07778E07B
:1011B000A79FD0011124942F907770E4979FF0019E
:1011C0001124EA2BFB2B5F77DF01A52BE22FE077C1
:1011D000F0E0FE2FEE27FF0FEA2BFB2B932F9F77DC
:1011E00030E0322F22273295330F307E292B677063
:1011F00090E8699FB0011124262B372B477050E0EF
:10120000542F4427550F550F242B352B9091560101
:10121000A92F092E000CBB0B2A9FA0012B9F500D5C
:101220003A9F500D112441386FEF560714F441E8EE
:101230005FEF51954195510941387FEF570714F4FD
:1012400041E85FEF419540935C01EA9FB001EB9F5D
:10125000700DFA9F700D112461385FEF750714F45B
:1012600061E87FEF71956195710961385FEF7507EE
:1012700014F461E87FEF619560935D01BF939F93E4
:10128000FF93EF93E62F062E000CFF0BFF936F9357
:101290003F932F93242F042E000C330B3F934F9337
:1012A0001F928F9380E492E09F938F930E947F061A
:1012B0008BE591E00E94511580915601482F082E30
:1012C000000C550B0FB6F894DEBF0FBECDBF2091BA
:1012D000120130911301283C310518F428E030E068
:1012E00002C024E030E091E0421753070CF090E098
:1012F000890F8093560128960FB6F894DEBF0FBE73
:10130000CDBFDF91CF911F910F91FF90EF90DF90B4
:10131000CF90BF90AF909F908F907F906F905F9095
:101320004F903F9008951F93CF93DF93C09100019A
:10133000D09101018FEF9FEF909301018093000105
:10134000CF3F8FEFD80709F074C08091540190917E
:1013500055010E949E220C9710F480E0BAC00E94B2
:101360008622909355018093540182E00E94170CCD
:10137000EC01892B09F05DC080917101882309F48B
:1013800058C087E00E94170C009709F452C09C01D6
:101390002F77332722303105A1F048F4211531058C
:1013A00069F02130310599F480788A641AC02330BD
:1013B000310551F02F373105A1F009C080788264E2
:1013C00010C0807889640DC0807888640AC08EE877
:1013D00091E09F938F930E947F060F900F9081E181
:1013E00078C0292F33272F7733272130310579F023
:1013F00050F02230310579F02330310581F49078B6
:10140000EC01D86416C09078EC01D26412C09078D8
:10141000EC01DA640EC09078EC01D9640AC08BE765
:1014200091E09F938F930E947F060F900F9080E131
:1014300050C08091620381FF18C0209709F48DCFBE
:1014400087E691E00E94E605DF93CF9382E691E084
:101450009F938F930E947F0680E691E00E94E605AD
:101460000F900F900F900F9003C0209709F475CF45
:10147000CF378FE7D80711F48FE705C0CF3F8FEF45
:10148000D80721F48FEF0E94880622C08D2F1C2FD1
:10149000DF3F11F48C2F1FEF90917001992359F0C9
:1014A000982F9F77923319F480788A6004C09A301D
:1014B00011F4807882630E9488061F3F49F0812FD3
:1014C00090E0982F88278F6F9093010180930001FF
:1014D00081E0DF91CF911F910895E82FF0E0E05A6D
:1014E000FE4F80810895682F609582E00C947C0CFB
:1014F00080916203816080936203569A5E9A0E9493
:101500006B0B2FEF83ED90E3215080409040E1F78B
:1015100000C000000E94A80682EC92E09F938F9387
:101520000E947F0663E082E00E94F40B99270F90EF
:101530000F908131910539F190F48730910519F1BF
:1015400038F49C01245031092230310500F51BC0CC
:1015500089309105C1F08D309105C9F414C08D31E9
:10156000910589F038F48431910569F0893191054C
:1015700071F409C0843C910531F0873C910519F064
:10158000813C910521F421E02093700102C010926A
:10159000700120917001211103C021E331E002C0EC
:1015A0002DE231E03F932F939F938F938AEA92E04D
:1015B0009F938F930E947F0663E087E00E94F40B65
:1015C000992721E00F900F900F900F900F900F90A0
:1015D0008230910509F020E020937101029741F4D7
:1015E0008EE992E09F938F930E947F060F900F9059
:1015F00023E042E063E082E00E94530CE0E6F1E089
:10160000119221E0E037F207D9F70E94FC140E9402
:10161000730A0E94A806569A5E980895509A83E02D
:1016200091E00197F1F700C0000050989AEB9A956D
:10163000F1F700C00895509A8AEB8A95F1F700C03F
:10164000509883E091E00197F1F700C00000089501
:10165000EF92FF920F931F93CF93DF93C0E0D0E000
:1016600090E8E92EF12C082F10E0C7010C2E02C0E3
:10167000959587950A94E2F780239123892B19F099
:101680000E941B0B02C00E940E0B2196C830D10590
:1016900061F7DF91CF911F910F91FF90EF90089527
:1016A000509A83EF9BE00197F1F700C000000C9483
:1016B0001B0B489B06C023E02A95F1F70000019719
:1016C000C1F70895489906C023E02A95F1F7000074
:1016D0000197C1F708955898509808950895EF928A
:1016E000FF920F931F93CF93DF93C82F162F7A018A
:1016F000D22F80E0422F50E0282F082E000C330B11
:101700002417350734F4F701E20FF31F10828F5FBF
:10171000F3CFF8940E94500B80E1C89F90011124F0
:10172000812F8C60822B0E94280B0E940E0B84EF6D
:1017300091E00E94620B892B19F482ED92E01AC0AD
:1017400084EF91E00E94590B892B19F4789480E082
:1017500044C088E290E00E94620B892B19F480ED6E
:1017600092E008C084E690E00E94590B892B51F466
:101770008EEC92E09F938F930E947F0678940F9057
:101780000F90E5CFC0E082E890E00E94620B8823D2
:10179000F9F08C011127C8010E94590B8823C1F070
:1017A0009C2F9695969596959D1780F4F701E90FD5
:1017B000F11D9081990F22E830E0201B310B081BAE
:1017C0001109201731070CF491609083CF5FD9F68F
:1017D00078948C2F869586958695DF91CF911F9171
:1017E0000F91FF90EF900895CF93DF93CDB7DEB7C1
:1017F00028970FB6F894DEBF0FBECDBF28E0AE012C
:101800004F5F5F4F0E946F0B823031F489819A8164
:1018100098278927982702C080E090E028960FB685
:10182000F894DEBF0FBECDBFDF91CF91089560E089
:101830000C94F40BEF92FF921F93CF93DF93D82F6A
:10184000162F7A01C22FF8940E94500B80E1D89F86
:1018500090011124812F8860822B0E94280B0E9406
:101860000E0B8FE193E00197F1F700C000000E949A
:101870001B0B10E0D0E0812F012E000C990B8C1770
:101880009D0744F4F701E80FF91F80810E94280B9F
:101890001F5FF1CF0E940E0B7894DF91CF911F91C3
:1018A000FF90EF900895CF93DF9300D0CDB7DEB7D0
:1018B00049832A8322E0AE014F5F5F4F0E941A0CDA
:1018C0000F900F90DF91CF910895CF93C82FF89488
:1018D0000E94500B20E1C29FC001112481600E9430
:1018E000280B0E940E0B8FE193E00197F1F700C0E7
:1018F00000007894CF910895262F277040E062E091
:101900000C94530C80917E020895CF93DF9300D006
:101910001F92CDB7DEB79C0180917703843019F513
:1019200093E099833B832A839093E9008FEF909112
:10193000E800815095FD06C095ED9A95F1F70000FD
:101940008111F5CF8091E80085FF0DC040E050E0A7
:1019500063E070E0CE0101960E94FC108091E800E7
:101960008E778093E8000F900F900F90DF91CF91CA
:101970000895CF93DF9300D01F92CDB7DEB72091AB
:101980007703243031F522E02983805891099B8325
:101990008A8383E08093E9008FEF9091E800815083
:1019A00095FD06C095ED9A95F1F700008111F5CFF0
:1019B0008091E80085FF0DC040E050E063E070E0FA
:1019C000CE0101960E94FC108091E8008E778093F2
:1019D000E8000F900F900F90DF91CF910895209124
:1019E00077032430F1F422E02093E9002FEF3091C7
:1019F000E800215035FD06C035ED3A95F1F70000BD
:101A00002111F5CF2091E80025FF0BC040E050E008
:101A100065E070E00E94FC108091E8008E77809372
:101A2000E8000895CF93DF9320917703243049F5A0
:101A300021E02093E90021E8215059F03091E8009D
:101A400035FD07C0EFE3F1E03197F1F700C000008A
:101A5000F3CF2091E80025FF14C0EC0140E050E0F6
:101A600068E070E00E94FC108091E8008E7780931F
:101A7000E80088E0FE01A6E7B2E001900D928A95A9
:101A8000E1F7DF91CF910895CF93C0917401C11117
:101A90000BC00E949222643C79408105910520F0A0
:101AA00081E080937401C1E08C2FCF910895FF9263
:101AB0000F931F93CF93DF93D82F0FB607FE83C0EA
:101AC00080917703843081F08091170190E0019636
:101AD0002091190130E0822393232091180130E0F6
:101AE0008217930709F0CDC00E94440D811110C0E8
:101AF0008091170190E001962091190130E0822336
:101B000093232091180130E08217930709F0B9C0A0
:101B10000E9486228C01C091E900CF709091EC0068
:101B2000892F817090FD80E8C82B84E08093E900C4
:101B300085E0F82E8091EB0085FD42C08091EB009E
:101B400080FF3EC08091EE0087FF3AC0809118016F
:101B500090911701981709F457C09091E80095FFEC
:101B60008EC0E0911501F0911601E80FF11D208162
:101B70008F5F909119018923809318012093F100C0
:101B80008091E80085FDE2CF8091E80080FFDECF04
:101B90008091E8008E778093E800F0921401D6CF10
:101BA0008091170190E001962091190130E0822385
:101BB00093232091180130E08217930709F44CC059
:101BC000CF70C093E90040911701842F90E00196F7
:101BD0002091190130E0822393232091180130E0F5
:101BE0008217930709F450C0E0911501F091160196
:101BF000E40FF11DD083809117018F5F909119013F
:101C000089238093170140C08091E80085FF37C089
:101C1000D093F10021E03091F3008091F20090E048
:101C2000932B892B91F08091E80080FF0EC080916A
:101C3000E80085FF03C01092F100F9CF8091E80021
:101C40008E778093E800F0921401222309F4A8CF44
:101C5000CF70C093E90018C080911401882309F463
:101C6000AFCF0E9486229C018017910711F4890151
:101C700061CF90911401915090931401F8CF20E01E
:101C8000CACF40911701B0CF80E0DF91CF911F9173
:101C90000F91FF90089580917603811109C00E94F1
:101CA00066130E94C3138091E20084608093E20077
:101CB00008951092760308950895089542E061EC26
:101CC00081E00E94751042E061EC82E00E94751094
:101CD00042E061EC83E00E94751042E261EC84E036
:101CE0000C94751080917903833009F453C030F45B
:101CF000813071F0823009F48CC008958A3009F483
:101D000078C08B3009F45EC0893009F09AC020C0D9
:101D100080917803813A09F094C08091E800877F30
:101D20008093E80080917C0390917D03892B21F4BE
:101D300068E086E792E003C060E080E090E070E059
:101D40000E9447118091E8008B778093E800089506
:101D500080917803813209F074C080917C03909166
:101D60007D03892B09F06DC08091E800877F809307
:101D7000E8008091E80082FD05C080917703811121
:101D8000F8CF5FC08091F10080937E028091E800DF
:101D90008B7753C080917803813A09F052C08091CB
:101DA0007C0390917D03892B09F04BC08091E80062
:101DB000877F8093E8008091E80080FFFCCF8091CE
:101DC000240136C0809178038132D9F580917C035B
:101DD00090917D03892BA9F58091E800877F8093FE
:101DE000E8000E94AA1080917A03809324010C9449
:101DF000341880917803813221F58091E800877F43
:101E00008093E8000E94AA1080917B0380937F0258
:101E1000089580917803813AA1F48091E800877F4A
:101E20008093E8008091E80080FFFCCF80917F02E2
:101E30008093F1008091E8008E778093E8000C9405
:101E4000AA10089580917E028093750110927E02FF
:101E50000E9465160C9434180C94220F0E941322D1
:101E600080917503882329F00E943C2281110C94F3
:101E70005F1008950E9450228091750180937E0228
:101E800008950C943A0F08950C94430F0C94430F4B
:101E9000CF9384B7877F84BF0FB6F894A8958091BD
:101EA0006000886180936000109260000FBE90E037
:101EB00080E80FB6F89480936100909361000FBEA4
:101EC00087E59DE00E94E6218AE191E00E94F714F7
:101ED00088EF92E00E94E6050E94460F0E94B61528
:101EE0000E9466130E94C3138091E2008460809375
:101EF000E20078940E94B81580917703843019F03D
:101F00000E94430FF9CF86EE92E00E94E6050E9400
:101F1000440F84ED92E00E94E605C4E080917703CF
:101F2000853019F40E942E0FF9CF0E94BE15209122
:101F3000E4003091E50080917201909173012817BF
:101F4000390761F38091E4009091E500909373016B
:101F5000809372010E94440D882301F380917703DE
:101F60008430E1F68091E9008F702091EC00922F8F
:101F7000917020FD90E8892BC093E9009091EB00CF
:101F800090FF43C09091EE0097FF3FC090911801E1
:101F900020911701291709F12091E80025FF1DC0A4
:101FA000E0911501F0911601E90FF11D30819F5F5D
:101FB000209119019223909318013093F100909190
:101FC000E80095FDE3CF9091E80090FFDFCF90917E
:101FD000E8009E779093E800D9CF9091F30020918C
:101FE000F20030E0392B232B81F09091E80090FF34
:101FF0000CC09091E80095FF03C01092F100F9CF5A
:102000009091E8009E779093E8008F708093E900AC
:1020100085CF292F332723303105C9F060F42130D3
:10202000310581F02230310509F041C084E790E0AC
:1020300023E533E040C021323105E1F022323105A1
:1020400031F135C082E190E027EC33E034C09927CC
:102050008130910549F028F0029749F5EFE0F3E06F
:1020600005C0EFE4F3E002C0EFE3F3E0849190E019
:102070009F0121C064307105D0F4660F771FFB010A
:10208000E05CFE4F2081318189E090E014C0643033
:10209000710568F4FB01EE0FFF1FE85CFE4F208125
:1020A0003181FB01EC5CFE4F808190E004C080E058
:1020B00090E020E030E0FA0131832083089580E150
:1020C00089BD82E189BD09B400FEFDCF8091D800B1
:1020D0008F7D8093D8008091E00082608093E00043
:1020E0008091E00081FDFCCF0895982F973068F52E
:1020F0009093E900981739F07091EC002091ED0071
:102100005091F00003C0242F762F50E021FD02C033
:102110009F5FECCF3091EB003E7F3093EB0030912E
:10212000ED003D7F3093ED003091EB003160309356
:10213000EB007093EC002093ED005093F0002091A1
:10214000EE0027FDE5CF80E008958F708093E900D1
:1021500081E008958091780387FF11C08091E800A5
:1021600082FD05C0809177038111F8CF11C0809165
:10217000E8008B770BC080917703882349F080912A
:10218000E80080FFF8CF8091E8008E778093E80028
:1021900008952091E4003091E50095E64091EC002F
:1021A000842F817040FF23C08091E80080FD1DC016
:1021B00080917703882399F0853099F08091EB0026
:1021C00085FD11C04091E4005091E50024173507CA
:1021D00029F3915011F09A01E1CF84E0089582E053
:1021E000089583E0089581E0089580E00895409186
:1021F000E80042FFDDCF0895CF92DF92EF92FF9289
:102200000F931F93CF93DF93EC018B017A010E9410
:10221000C910811133C0E114F10439F0F701808154
:102220009181081B190BC80FD91FC12CD12C011586
:10223000110519F18091E80085FD16C08091E80034
:102240008E778093E800E114F10449F0F701808172
:102250009181C80ED91ED182C08285E00FC00E9434
:10226000C910882321F30AC089918093F10001509D
:102270001109FFEFCF1ADF0ADACF80E0DF91CF91AB
:102280001F910F91FF90EF90DF90CF9008952091D4
:102290007E0330917F032617370748F061157105DB
:1022A00039F42091E8002E772093E80001C0B901AD
:1022B000FC0120E06115710579F180917703882395
:1022C000F1F18530F1F18091E80083FD3CC080910F
:1022D000E80082FD2EC08091E80080FFEBCF2091C6
:1022E000F3008091F20090E0922B6115710551F09E
:1022F0008830910538F421912093F10061507109E3
:102300000196F3CF21E0089709F020E08091E800E2
:102310008E778093E800CECF2111CFCF0AC0809175
:102320007703882361F0853061F08091E80083FDB8
:102330000AC08091E80082FFF2CF80E0089582E039
:10234000089583E0089581E0089520917E033091FF
:102350007F032617370748F06115710539F420917E
:10236000E8002E772093E80001C0B901FC0120E0CD
:102370006115710591F180917703882309F440C0BC
:10238000853009F43FC08091E80083FD3DC0809115
:10239000E80082FD2FC08091E80080FFE9CF209106
:1023A000F3008091F20090E0922B6115710559F0D5
:1023B0008830910540F424912093F10031966150CA
:1023C00071090196F2CF21E0089709F020E0809191
:1023D000E8008E778093E800CBCF2111CCCF0AC0E4
:1023E00080917703882361F0853061F08091E80067
:1023F00083FD0AC08091E80082FFF2CF80E008955B
:1024000082E0089583E0089581E008951F93CF93BB
:10241000DF93CDB7DEB7AA970FB6F894DEBF0FBE35
:10242000CDBFE8E7F3E08091F100819323E0E0384D
:10243000F207C9F70E94720E8091E80083FF2EC157
:102440008091780390917903492F50E04A305105EB
:1024500008F024C1FA01EA5AFF4F0C94062B803889
:1024600021F0823809F01AC108C08091740390915C
:102470007503992389F082600FC080917C038F706F
:10248000873008F00BC18093E9008091EB0085FB59
:10249000882780F91092E9009091E800977F909347
:1024A000E8008093F1001092F100D1C0282F2D7F19
:1024B00009F0F4C0882319F0823061F0EFC08091F8
:1024C0007A03813009F0EAC0933009F080E080930C
:1024D00075032EC080917A0381112AC080917C03FC
:1024E0008F702FEF280F263008F0D8C08093E900B6
:1024F0002091EB0020FF1CC0933021F48091EB0071
:10250000806214C09091EB0090619093EB0021E009
:1025100030E0A90102C0440F551F8A95E2F74093AD
:10252000EA001092EA008091EB0088608093EB0053
:102530001092E9008091E800877F8093E8000E9474
:10254000AA10ACC08111AAC010917A031F778091A4
:10255000E3008078812B8093E3008091E800877FFF
:102560008093E8000E94AA108091E80080FFFCCFD1
:102570008091E30080688093E300111102C082E043
:1025800001C083E08093770389C08058823008F0CF
:1025900085C080917A0390917B038C3D53E0950731
:1025A00079F583E08A838AE289834FB7F894DE0164
:1025B000139620E03EE051E2E32FF0E05093570005
:1025C000E49120FF03C0E295EF703F5FEF708E2F24
:1025D00090E0EA3010F0C79601C0C0968D939D93AD
:1025E0002F5F243149F74FBF8091E800877F8093A8
:1025F000E8006AE270E0CE0101960E94471116C021
:1026000060917C0370917D03AE014F5F5F4F0E942C
:102610000910BC01892B09F441C09091E800977F13
:102620009093E80089819A810E94A5118091E80029
:102630008B778093E80032C0803881F58091E80084
:10264000877F8093E800809173038093F1008091ED
:10265000E8008E7772CF811121C080917A0390912A
:102660007B0399270297D4F48091E800877F8093B9
:10267000E80080917A03809373030E94AA108091EE
:102680007303811106C08091E30087FD02C081E0E1
:1026900001C084E0809377030E945E0E8091E80081
:1026A00083FF0AC08091E800877F8093E8008091D3
:1026B000EB0080628093EB00AA960FB6F894DEBF21
:1026C0000FBECDBFDF91CF911F9108950E94D4130B
:1026D0000E94DC13E0EEF0E0808181608083E8ED11
:1026E000F0E080818F77808319BCA7EDB0E08C91FA
:1026F0008E7F8C9380818F7E8083109276030895E5
:102700000F931F93CF93DF930E94D4130E94DC1387
:10271000C8EDD0E088818F7788838881806888833E
:1027200088818F7D888319BC109277031092730380
:10273000109275031092740300EE10E0F80180818E
:102740008B7F808388818160888342E060E080E0C5
:102750000E947510E1EEF0E080818E7F8083E2EED2
:10276000F0E0808181608083808188608083F801CF
:1027700080818E7F8083888180618883DF91CF9183
:102780001F910F910895E8EDF0E080818F7E8083A6
:10279000E7EDF0E080818160808384E082BF81E0AA
:1027A000809376030C948013E8EDF0E080818E7FB7
:1027B00080831092E20008951092DA001092E100F6
:1027C00008951F920F920FB60F9211242F933F93EB
:1027D0004F935F936F937F938F939F93AF93BF9329
:1027E000EF93FF938091E10082FF0BC08091E200A4
:1027F00082FF07C08091E1008B7F8093E1000E94FF
:102800005D0E8091DA0080FF1FC08091D80080FFAC
:102810001BC08091DA008E7F8093DA008091D9000E
:1028200080FF0DC080E189BD82E189BD09B400FE51
:10283000FDCF81E0809377030E944B0E05C019BC49
:10284000109277030E94590E8091E10080FF19C019
:102850008091E20080FF15C08091E2008E7F80931E
:10286000E2008091E20080618093E2008091D800D4
:1028700080628093D80019BC85E0809377030E9422
:102880002C0F8091E10084FF30C08091E20084FF32
:102890002CC080E189BD82E189BD09B400FEFDCF75
:1028A0008091D8008F7D8093D8008091E1008F7E49
:1028B0008093E1008091E2008F7E8093E20080911E
:1028C000E20081608093E20080917303882311F01D
:1028D00084E007C08091E30087FD02C081E001C071
:1028E00083E0809377030E94410F8091E10083FF92
:1028F00029C08091E20083FF25C08091E100877F9D
:102900008093E10082E080937703109273038091BB
:10291000E1008E7F8093E1008091E2008E7F8093C2
:10292000E2008091E20080618093E20042E060E09A
:1029300080E00E9475108091F00088608093F00024
:102940000E945C0EFF91EF91BF91AF919F918F918B
:102950007F916F915F914F913F912F910F900FBE9B
:102960000F901F9018951F920F920FB60F9211247F
:102970002F933F934F935F936F937F938F939F9387
:10298000AF93BF93CF93DF93EF93FF93C091E90091
:10299000CF708091EC00D82FD17080FDD0E81092DC
:1029A000E9008091F000877F8093F00078940E9486
:1029B00006121092E9008091F00088608093F00088
:1029C000CD2BCF70C093E900FF91EF91DF91CF91B4
:1029D000BF91AF919F918F917F916F915F914F9137
:1029E0003F912F910F900FBE0F901F9018959093CD
:1029F0008502809384020895E0918402F09185021B
:102A0000309721F00190F081E02D099480E0089545
:102A1000EF92FF920F931F93CF93DF93E091840285
:102A2000F09185023097B1F18C010280F381E02DA5
:102A300009958091620382FF2DC080FF04C084EE5F
:102A400094E00E94E605E80118E08EEDE82E84E0AF
:102A5000F82E8091620380FF0BC088811F928F93B4
:102A6000FF92EF920E947F060F900F900F900F90B1
:102A7000115021961111EDCF8091620380FF0AC0A1
:102A80008CED94E0DF91CF911F910F91FF90EF902B
:102A90000C94E605DF91CF911F910F91FF90EF907D
:102AA0000895E0918402F0918502309721F004802E
:102AB000F581E02D09940895CF93DF932091820250
:102AC000309183022817390709F19093830280938C
:102AD0008202E0918402F09185023097B9F0EC0116
:102AE0000680F781E02D09958091620382FF0EC078
:102AF00080FF0CC0DF93CF938EEC94E09F938F9375
:102B00000E947F060F900F900F900F90DF91CF9152
:102B10000895CF93DF93209180023091810228178E
:102B2000390709F19093810280938002E091840239
:102B3000F09185023097B9F0EC010084F185E02D29
:102B400009958091620382FF0EC080FF0CC0DF9365
:102B5000CF938EEB94E09F938F930E947F060F900C
:102B60000F900F900F90DF91CF9108950C946616FF
:102B70000E947D220E94780A0C946E0BBF92CF9225
:102B8000DF92EF92FF920F931F93CF93DF9300D0CA
:102B900000D01F92CDB7DEB70E94930907E812E07C
:102BA000F12C8F2D0E946D0AB82EF801C080C82626
:102BB00039F4F3940F5F1F4FF0E1FF12F2CF30C0F2
:102BC0008091620381FD0E947B16D12CEE24E39458
:102BD0008C2D8E21F9F0D982FA8291E08B2D8E21F5
:102BE00009F490E09B830E9486228160782F9D8368
:102BF0008C8349815A816B818D810E94B1164981F4
:102C00005A816B817C818D810E94FE21F801808137
:102C10008E258083D394EE0CF8E0DF12D9CFC9CF94
:102C20008FEF89838A831B820E9486228160782F9E
:102C30009D838C8349815A816B818D810E94B1165D
:102C40000E94FD210E9444250E94D5060E94FC148A
:102C500090918602891741F10E94FC1480938602AC
:102C60009091620392FF0EC090FF0CC01F928F9351
:102C70008FEE94E09F938F930E947F060F900F90AA
:102C80000F900F90809186020F900F900F900F90F1
:102C90000F90DF91CF911F910F91FF90EF90DF90F8
:102CA000CF90BF900C940F220F900F900F900F9029
:102CB0000F90DF91CF911F910F91FF90EF90DF90D8
:102CC000CF90BF9008950C94730A08950895CF9300
:102CD000C62F0E946D0A21E030E002C0220F331F90
:102CE000CA95E2F790E02823392381E0232B09F4E9
:102CF00080E0CF910895EF92FF920F931F93CF93AF
:102D0000DF9388E095E00E94E605C0E0D0E083E331
:102D1000E82E81E0F82E0AEF14E08C2F0E946D0A55
:102D20000E94EB21FF92EF921F928F93DF93CF933C
:102D30001F930F930E947F0621968DB79EB708962A
:102D40000FB6F8949EBF0FBE8DBFC031D10529F7D5
:102D5000DF91CF911F910F91FF90EF90089508950B
:102D60000895CF93DF93CDB7DEB72B970FB6F894C6
:102D7000DEBF0FBECDBF942F4F83252F58876987A5
:102D80007A878B874A855B85452B31F02F3F31F45D
:102D900081E09F3F19F403C081E001C080E080FD25
:102DA00007C04F81588569857A858B850E94FE21F1
:102DB000DE01119686E0FD0111928A95E9F785E022
:102DC000FE01379601900D928A95E1F749815A816B
:102DD0006B817C818D819E810E94601E2B960FB637
:102DE000F894DEBF0FBECDBFDF91CF910895CF9392
:102DF000882309F4A9C0C82F8238A1F40E94FC14CA
:102E000081FDA2C089E30E9448210E94C0212FEFCA
:102E100081EE94E0215080409040E1F700C0000036
:102E200089E315C08338C1F40E94FC1480FD8CC076
:102E300083E50E9448210E94C0212FEF81EE94E09B
:102E4000215080409040E1F700C0000083E50E94DF
:102E50006521CF910C94C0218438A1F40E94FC1408
:102E600082FD72C087E40E9448210E94C0212FEF9A
:102E700081EE94E0215080409040E1F700C00000D6
:102E800087E4E5CF8CEF8C0F813A20F080E58C0F42
:102E90008E3248F48C2F0E946E28811155C08C2FE1
:102EA0000E944821D6CF80E28C0F883048F4C7704A
:102EB00081E001C0880FCA95EAF70E948621C9CF38
:102EC0008BE58C0F833078F4C53A29F0C63A31F09F
:102ED00083E890E005C081E890E002C082E890E0DD
:102EE000CF910C945C1588E58C0F853168F5C83A54
:102EF00089F0C93A91F0CA3A99F0CB3AA1F0CC3AAC
:102F0000A9F0CD3AB1F0CE3AB9F0CF3AC1F080E0B5
:102F100090E017C082EE90E014C089EE90E011C0FE
:102F20008AEE90E00EC085EB90E00BC086EB90E05F
:102F300008C083EB90E005C084EB90E002C087EB13
:102F400090E0CF910C948915CF910895882309F4CE
:102F50006AC08238A1F40E94FC1481FF64C089E336
:102F60000E9448210E94C0212FEF81EE94E0215061
:102F700080409040E1F700C0000089E315C083382D
:102F8000B9F40E94FC1480FF4EC083E50E944821E2
:102F90000E94C0212FEF81EE94E0215080409040AC
:102FA000E1F700C0000083E50E9465210C94C02178
:102FB0008438A1F40E94FC1482FF35C087E40E948B
:102FC00048210E94C0212FEF81EE94E021508040E3
:102FD0009040E1F700C0000087E4E6CF9CEF980F37
:102FE000913A10F390E5980F9E32F0F290E2980F2C
:102FF000983050F4877091E001C0990F8A95EAF7F4
:10300000892F0E948C21D2CF9BE5980F933020F41A
:1030100080E090E00C945C15885A853120F480E0C3
:1030200090E00C9489150895882321F00E94862150
:103030000C94C0210895882321F00E948C210C94C7
:10304000C02108950E94A6210E9475210E94C021DE
:103050000E94E9250E94B72480E090E00E945C1560
:1030600080E090E00C9489150E9496210C9422181F
:10307000CF92DF92EF92FF920F931F93CF93DF9344
:1030800000D000D01F92CDB7DEB76C010E94112294
:10309000811101C385E0F601DE01119601900D92C8
:1030A0008A95E1F7F6014081518123813481211510
:1030B000310531F05F3F31F481E04F3F19F403C037
:1030C00081E001C080E080FDE6C2F601F280E5808B
:1030D000E2948FE0E82249835A83FB82722F3D837A
:1030E0002C836F2D8D810E94C4208C010E94C320EF
:1030F0000E94B31FE12FE295EF708E2F90E0FC014C
:10310000E05AFF4F0C94062B812F807F1F7088237D
:1031100011F01295107FFF2049F0112309F452C2DB
:10312000812F0E9499210E94C0214CC2802F0E94B1
:10313000A617112309F4AFC2812F0E949F210F907F
:103140000F900F900F900F90DF91CF911F910F91E3
:10315000FF90EF90DF90CF900C94C021812F807F63
:103160001F70803211F01295107F002319F001308A
:1031700009F12BC0FF20A9F0EE2059F1F1E0812FD9
:10318000EF1228C00F900F900F900F900F90DF91CB
:10319000CF911F910F91FF90EF90DF90CF900C9403
:1031A000A921EE2021F021E0E21609F474C20E9468
:1031B000AC212DC0FF20E9F085E08E1508F46BC22C
:1031C0000E948321812329F022C0FF20F1F0E11029
:1031D00015C0812F0F900F900F900F900F90DF91DF
:1031E000CF911F910F91FF90EF90DF90CF900C94B3
:1031F000141894E09E1508F44EC209C0F6018581AA
:1032000080FFE0C18F708583E4CFE110EEC1812F94
:1032100061C1812F86958695837019F08130B9F050
:103220003AC2FF2019F0C801937002C080E090E01C
:103230000F900F900F900F900F90DF91CF911F91F3
:103240000F91FF90EF90DF90CF900C945C15FF20D2
:1032500019F0C801937002C080E090E00F900F90C9
:103260000F900F900F90DF91CF911F910F91FF90D2
:10327000EF90DF90CF900C948915802FFF2019F0EC
:103280000E94CA2302C00E9432240F900F900F9018
:103290000F900F90DF91CF911F910F91FF90EF90C2
:1032A000DF90CF900C94B724812F837009F070C009
:1032B000F110F1C1202F229526952770220F220FA1
:1032C000602F6F70862F90E0A0E0B0E06C017D0170
:1032D000022E04C0CC0CDD1CEE1CFF1C0A94D2F79D
:1032E00004FF12C08FE090E0A0E0B0E004C0880FBF
:1032F000991FAA1FBB1F2A95D2F7BC01CD0160956B
:1033000070958095909503C060E070E0CB011695B4
:10331000169513701230B1F040F56C297D298E2975
:103320009F29113031F10F900F900F900F900F9057
:10333000DF91CF911F910F91FF90EF90DF90CF9091
:103340000C94D81F6C297D298E299F290F900F90EE
:103350000F900F900F90DF91CF911F910F91FF90E1
:10336000EF90DF90CF900C94F21F0E94D81FC701FE
:10337000B6010F900F900F900F900F90DF91CF91AB
:103380001F910F91FF90EF90DF90CF900C94BE1F94
:10339000FF2019F0812F817001C08695882309F4E0
:1033A0007AC1202F229526952770220F220F602F99
:1033B0006F70862F90E0A0E0B0E06C017D01022EDE
:1033C00004C0CC0CDD1CEE1CFF1C0A94D2F704FFD9
:1033D00012C08FE090E0A0E0B0E004C0880F991F19
:1033E000AA1FBB1F2A95D2F7BC01CD01609570952D
:1033F0008095909503C060E070E0CB01169516951E
:1034000013701230B1F040F56C297D298E299F2967
:10341000113031F10F900F900F900F900F90DF91BE
:10342000CF911F910F91FF90EF90DF90CF900C9470
:103430009F206C297D298E299F290F900F900F9036
:103440000F900F90DF91CF911F910F91FF90EF9010
:10345000DF90CF900C94B1200E949F20C701B6014D
:103460000F900F900F900F900F90DF91CF911F91C1
:103470000F91FF90EF90DF90CF900C948D20003F44
:10348000C1F128F480E4800F803250F096C0023FF2
:1034900009F45EC008F449C0033F09F46CC08DC054
:1034A000F02FF071EF2E812F8F71FF2051F00E94CD
:1034B0002620802FEE2019F08295807F8BCE8F7092
:1034C00089CE0E944720802FEE2019F08295807FC0
:1034D00001C08F700F900F900F900F900F90DF91A1
:1034E000CF911F910F91FF90EF90DF90CF900C94B0
:1034F0001B18FF20A9F024E02E1508F4CCC0812F62
:103500008F710F900F900F900F900F90DF91CF91D0
:103510001F910F91FF90EF90DF90CF900C946C2053
:1035200085E08E1508F4B7C0EACFFF2099F0812F0F
:103530008F710F900F900F900F900F90DF91CF91A0
:103540001F910F91FF90EF90DF90CF900C94262069
:10355000FF2069F3812F8F710F900F900F900F90C4
:103560000F90DF91CF911F910F91FF90EF90DF901F
:10357000CF900C944720FF2089F0812F8F710F90FE
:103580000F900F900F900F90DF91CF911F910F919F
:10359000FF90EF90DF90CF900C9411200F900F9040
:1035A0000F900F900F90DF91CF911F910F91FF908F
:1035B000EF90DF90CF900C940C20FF2099F0EE203C
:1035C00009F4B5CF802F0F900F900F900F900F90B0
:1035D000DF91CF911F910F91FF90EF90DF90CF90EF
:1035E0000C94F716EE2009F4B5CF802F0F900F90B2
:1035F0000F900F900F90DF91CF911F910F91FF903F
:10360000EF90DF90CF900C94A617412F4F70602F52
:10361000C6010E9444230F900F900F900F900F90BF
:10362000DF91CF911F910F91FF90EF90DF90CF909E
:103630000C940E1F01112FC0FF2069F10E94341855
:103640009FEFE0E7F2E09150E040F040E1F700C08A
:1036500000000F900F900F900F900F90DF91CF917F
:103660001F910F91FF90EF90DF90CF900C94ED227F
:10367000412F4F70602FC6010F900F900F900F9049
:103680000F90DF91CF911F910F91FF90EF90DF90FE
:10369000CF900C9447230F900F900F900F900F90A6
:1036A000DF91CF911F910F91FF90EF90DF90CF901E
:1036B00008951F93CF93DF9300D000D01F92CDB712
:1036C000DEB7942F4983252F5A836B837C838D83A8
:1036D0004C815D81452B31F02F3F31F481E09F3FDC
:1036E00019F403C081E001C080E0182F117080FD43
:1036F00031C049815A816B817C818D810E94C420B7
:10370000292F22952F702C3030F42A30A0F422502B
:10371000223030F022C02C30C9F02F30B9F01DC05B
:10372000853A28F48430C0F4823028F415C090E241
:10373000980F983088F0883E30F4803E68F48450CA
:10374000813A58F409C0803F41F406C093FB112729
:1037500010F903C010E001C011E0812F0F900F900D
:103760000F900F900F90DF91CF911F910895CF93FD
:10377000DF9300D000D01F92CDB7DEB70F900F902F
:103780000F900F900F90DF91CF910895CF93DF931B
:1037900000D000D000D0CDB7DEB726960FB6F89493
:1037A000DEBF0FBECDBFDF91CF9108951F93CF93A2
:1037B000DF93C091970216E080919802C81799F0A4
:1037C000D0E01C9FF0011D9FF00D1124E756FD4F26
:1037D0004081518162817381848195810E94C61BE1
:1037E0002196C770E9CFDF91CF911F910895409145
:1037F000C9025091CA026091CB027091CC028091B3
:10380000CD029091CE020C94C61BCF938091CE0234
:1038100082958F7009F05FC08091CB02882309F4F4
:103820005AC080919702B09198027091C902A091FC
:10383000CA024091CC025091CD0291E07F3F09F045
:1038400090E0692FC6E08B1709F445C0411551057A
:1038500021F0AF3F21F020E003C021E001C0262F7E
:1038600090E020FD35C0C89FF001C99FF00D1124E4
:10387000E756FD4F21812A132BC02081271328C032
:103880002281211125C0238134812417350710F4AA
:1038900021503109241B350B283C3105C8F42091F7
:1038A000CE022F7020612093CE0226E0289FF001E7
:1038B000299FF00D1124E256FD4F80818F708061A9
:1038C000808389EC92E00E943818CF910C94D61B2B
:1038D00001968770B8CFCF910895AF92BF92CF92E3
:1038E000DF92EF92FF920F931F93CF93DF93CDB7A9
:1038F000DEB761970FB6F894DEBF0FBECDBF7C0177
:1039000085E0F701DE011D9601900D928A95E1F7A1
:10391000D7014C9111965C9111971296DC901297F9
:1039200013960D911C9114973091C9026091CA02AF
:103930008091CC029091CD02009731F06F3F31F42D
:1039400021E03F3F19F403C021E001C020E0B22F85
:10395000B170BB2E20FD6EC1A090CB02AA2009F44D
:10396000CCC02091CE020817190728F0F801E81BF7
:10397000F90BCF0104C080959095800F911FCC2446
:10398000C394883C910580F0C12C207F09F0A1C030
:10399000702F198B088B6D2D89890E94B71B89ECBC
:1039A00092E00E943818BDC0822F807F09F056C077
:1039B000561315C0431313C0CD2CD11010C02F7057
:1039C00020612093CE020E94F71B89EC92E00E94B6
:1039D00038188091CE02D70115968C935FC10115DE
:1039E000110531F05F3F31F481E04F3F19F403C01E
:1039F00081E001C080E080FD03C081E08D2502C030
:103A000080E090E0B82FB170CB2E80FF1CC0809179
:103A100097022091980236E0821709F41CC190E0C9
:103A2000389FF001399FF00D1124E756FD4F618159
:103A3000561306C06081461303C06281D61203C0CC
:103A400001968770E9CFCD2CDD2009F427C1809144
:103A5000CE0281608093CE02C12C20C1561308C0D3
:103A6000431306C0D11004C08091CE02D701B6C066
:103A70004D875E87DF86702F198B088B6D2D8989A6
:103A80000E94591B882399F1DD2089F12091CE02F3
:103A9000822F82958F7090E0029774F08091C90216
:103AA0009091CA0298878F8319861B870A872C8773
:103AB000CE0107960E94381886E0F701A9ECB2E023
:103AC00001900D928A95E1F70E94051C0E94F71B58
:103AD00011C0561781F14D875E87DF86702F198BD5
:103AE000088B6D2D89890E94591B811138C0C7012F
:103AF0000E943818CC24C394D1C00817190708F4C1
:103B000046C0F801E81BF90BCF01883C910508F489
:103B100043C0C12C702F198B088B6D2D89890E9491
:103B2000B71BE9ECF2E086E0DF011D928A95E9F728
:103B30000E94F71BB3C04313CECFD110CCCF8091DE
:103B4000CE02F7018583C7010E94381886E0E9ECB0
:103B5000F2E0DF011D928A95E9F7CA2C9FC0DD20B3
:103B600031F22091CE02822F82958F7090E00297E1
:103B70000CF4A2CF8091C9029091CA029A838983E2
:103B80001B821D830C832E83CE01019693CF8095DB
:103B90009095800F911FB9CFCD2CDD2009F4A7CFD0
:103BA000561333C0431331C02091CE0220FD24C0F0
:103BB000822F82958F70482F50E041155105E1F01A
:103BC000D70115962C9315974F30510549F08F5F0B
:103BD000982F9295907F822F8F70892B15968C93BA
:103BE000C7010E94381886E0F701A9ECB2E0019005
:103BF0000D928A95E1F79CCF86E0F701A9ECB2E03F
:103C000001900D928A95E1F749C04D875E87DF8666
:103C1000702F198B088B6D2D89890E94591B81117A
:103C20004BCF8091CE0281608093CE02C7010E946B
:103C3000381834C0DD2009F45ACF4D875E87DF86FF
:103C4000702F198B088B6D2D89890E94591B882331
:103C500009F44DCF31CF702F198B088B6D2D8989C9
:103C60000E94C420292F22952F70223028F49F70A3
:103C700039F0811105C00BC0243028F49F7049F43D
:103C8000805E883020F0C7010E943818BC2CCB2CF5
:103C900005C0F7019581907F99F7F9CF8C2D61963A
:103CA0000FB6F894DEBF0FBECDBFDF91CF911F914D
:103CB0000F91FF90EF90DF90CF90BF90AF9008955D
:103CC0001F93CF93DF93CDB7DEB72C970FB6F89441
:103CD000DEBF0FBECDBF4F83588769877A878B873A
:103CE0009C87CE0107960E946D1C8823D1F09F818E
:103CF00088852A853B85232B31F08F3F31F481E085
:103D00009F3F19F403C081E001C080E080FD47C0FF
:103D10004F81588569857A858B859C850E94C61B55
:103D20003EC086E0FE013796DE01119601900D92AD
:103D30008A95E1F7FF81E8856A857B8561157105C4
:103D400031F0EF3F31F481E0FF3F19F403C081E02F
:103D500001C080E080FD23C02091980230E0C901BD
:103D60000196877099274091970250E08417950734
:103D7000F1F1F983EA837D836C8396E0929FD00111
:103D8000939FB00D1124A756BD4FFE0131960190AF
:103D90000D929A95E1F7809398020E94D61B16E047
:103DA0008091970290919802891771F1189FC00134
:103DB000112487569D4F0E946D1C882329F1E091A4
:103DC00097021E9FF0011124E756FD4F408151815B
:103DD00062817381848195810E94C61B80919702C4
:103DE00090E001968770992780939702D9CF0E941F
:103DF00034181092980210929702E9ECF2E086E0F3
:103E0000DF011D928A95E9F72C960FB6F894DEBF74
:103E10000FBECDBFDF91CF911F910895DF92EF923A
:103E2000FF920F931F93CF93DF93FC01892B09F42B
:103E300088C0E12CF12CDD24D394EF0121968491EC
:103E4000853709F460C058F4843708F04EC08430D8
:103E500008F068C08130D1F0823071F172C08837CB
:103E600009F45BC050F4863709F453C0873709F072
:103E700068C08E2D0E94932152C09CE7980F903706
:103E800008F05FC08F770E94A6174EC08F010E5FAB
:103E90001F4FFE01849190E2980F983050F4877084
:103EA000FD2D01C0FF0F8A95EAF78F2F0E949921FF
:103EB00015C00E94F71614C08F010E5F1F4FFE0140
:103EC000849190E2980F983068F48770FD2D01C0BE
:103ED000FF0F8A95EAF78F2F0E949F210E94C02131
:103EE000E80122C00E94A617FBCFCF010296FE0177
:103EF000C491CC2361F0EFE9FFE03197F1F700C006
:103F00000000C150F6CFCF010296FE01F490EC0103
:103F10000BC00E948321E82E07C00E9496210E94B8
:103F2000C02102C00E94F7168F2D882341F0EFE9CF
:103F3000FFE03197F1F700C000008150F6CFFE019D
:103F40007CCFDF91CF911F910F91FF90EF90DF9089
:103F5000089560934F03709350038093510390939F
:103F600052030C940E2208956093530370935403EC
:103F700080935503909356030C940D220F931F9337
:103F8000009153031091540320915503309156032F
:103F9000602B712B822B932B6093530370935403EC
:103FA00080935503909356031F910F910C940D220B
:103FB0000F931F93009153031091540320915503C5
:103FC000309156036023712382239323609353031C
:103FD0007093540380935503909356031F910F9150
:103FE0000C940D220F931F930091530310915403CF
:103FF000209155033091560360277127822793271C
:104000006093530370935403809355039093560326
:104010001F910F910C940D2260E070E0CB010C9485
:10402000A91F0F931F9341E050E060E070E08A0108
:104030009B0104C0000F111F221F331F8A95D2F766
:10404000C901B8011F910F910C94A91F0F931F93E1
:1040500041E050E060E070E004C0440F551F661F6F
:10406000771F8A95D2F780914F0390915003A091CA
:104070005103B09152038A019B01082B192B2A2B63
:104080003B2BC901B8011F910F910C94A91F0F93ED
:104090001F9341E050E060E070E004C0440F551F02
:1040A000661F771F8A95D2F7409550956095709559
:1040B00080914F0390915003A0915103B09152030E
:1040C0008A019B01082319232A233B23C901B80134
:1040D0001F910F910C94A91F0F931F9341E050E083
:1040E00060E070E004C0440F551F661F771F8A957B
:1040F000D2F780914F0390915003A0915103B0915A
:1041000052038A019B01082719272A273B27C90147
:10411000B8011F910F910C94A91F0F931F93009149
:104120004F03109150032091510330915203602BA3
:10413000712B822B932B1F910F910C94A91F0F931E
:104140001F9300914F031091500320915103309120
:10415000520360237123822393231F910F910C94A8
:10416000A91F0F931F9300914F03109150032091AB
:1041700051033091520360277127822793271F91A3
:104180000F910C94A91F08958F929F92AF92BF92A6
:10419000DF92EF92FF920F931F93CF93DF9300D0A4
:1041A00000D01F92CDB7DEB76B837C838D838A01ED
:1041B0008C819D81892B31F01F3F31F481E04F3F8D
:1041C00019F403C081E001C080E080FF03C080E0FB
:1041D00090E04DC08B818823D1F180904F03909067
:1041E0005003A0905103B0905203809153039091DB
:1041F0005403A0915503B0915603882A992AAA2AFC
:10420000BB2A8FE1E82EF12CD501C4010E2C04C08D
:10421000B695A795979587950A94D2F780FD06C025
:1042200081E0E81AF10880F7D12C07C0DE2CB80134
:104230008E2D0E941C23019799F388E0189FF001AE
:104240001124E153FD4FE00FF11DD08209C088E039
:10425000189FF0011124E153FD4FE00FF11DD080B4
:1042600009831A8369817A818D2D0E941C230F9006
:104270000F900F900F900F90DF91CF911F910F91A2
:10428000FF90EF90DF90BF90AF909F908F90089538
:104290002091250130912601F90132969FEF40E0EF
:1042A0005191851789F09F3F19F4511101C0942F46
:1042B0004F5F4630A9F79F3F39F0F901E90FF11D33
:1042C00097FDFA95828308950895E0912501F09174
:1042D00026019F012A5F3F4F9281891301C01282FC
:1042E0003196E217F307C1F7089581E090E0E0917D
:1042F0002501F0912601E80FF91F10820196883000
:104300009105A9F708958091610308959091610343
:10431000892B80936103089580959091610389238F
:10432000809361030895809361030895109261035F
:10433000089590916003892B809360030895809580
:104340009091600389238093600308951092600325
:10435000089580935703089510925703089580910C
:10436000250190912601FC0131969C01285F3F4F69
:1043700080E0919191118F5FE217F307D1F70895D3
:10438000E0912501F0912601809161038083E09105
:104390002501F0912601908180916003892B808313
:1043A00080915703882361F0E0912501F091260167
:1043B0009081892B80830E94AF2181111092570335
:1043C00080912501909126010C940815909353013A
:1043D0008093520108958295982F937344E0949F9F
:1043E000900111248C7C86958695282B822F8575CB
:1043F000880F2A7A2695822B08950895CF93DF930C
:1044000000D000D01F92CDB7DEB70F900F900F9065
:104410000F900F90DF91CF910895089508950C9417
:10442000631680E0089580917703843021F1109223
:10443000630320E488E190E00FB6F894A895809398
:1044400060000FBE2093600083B7817F846083BFCC
:1044500083B7816083BF7894889583B78E7F83BF4D
:104460000FB6F894A89580916000886180936000F1
:10447000109260000FBE0895CF930E94AF160E9465
:1044800093090E94B016C0E08C2F0E946D0A811122
:1044900004C0CF5FC031C1F701C081E0CF91089562
:1044A0000E9465160C9434181F920F920FB60F924B
:1044B00011248F939F93AF93BF93809163038111D6
:1044C00013C08091640390916503A0916603B0913D
:1044D00067034196A11DB11D80936403909365030A
:1044E000A0936603B0936703BF91AF919F918F91A3
:1044F0000F900FBE0F901F90189582E084BD93E03F
:1045000095BD9AEF97BD80936E0008952FB7F894EC
:104510008091640390916503A0916603B091670355
:104520002FBF08952FB7F8946091640370916503CD
:1045300080916603909167032FBF0895CF92DF9219
:10454000EF92FF920F931F932FB7F894409164035B
:104550005091650360916603709167032FBF6A01F4
:104560007B01EE24FF248C0120E030E0C016D10650
:10457000E206F30610F4415051099A01281B390B49
:10458000C9011F910F91FF90EF90DF90CF90089598
:104590001F920F920FB60F9211248F939F93AF9398
:1045A000BF938091640390916503A0916603B091DD
:1045B00067030196A11DB11D809364039093650369
:1045C000A0936603B0936703BF91AF919F918F91C2
:1045D0000F900FBE0F901F9018950E946613F894CD
:1045E00087E797E7909301088093000887E090EBB6
:1045F000DC018093800390938103A0938203B093A6
:1046000083039CE088E10FB6F894A895809360003E
:104610000FBE90936000FFCFE82FF0E088E0989FF6
:10462000E00DF11D1124E052FF4F8491982F9295D7
:104630009F708F7097700895CF93C82FCB010E9401
:104640000C2340E1949F90011124282B2038310540
:104650001CF080E090E016C09770E92FF0E098E041
:10466000C99FE00DF11D112494E0EE0FFF1F9A95F4
:10467000E1F78F70E80FF11DEE0FFF1FE050F849D2
:1046800085919491CF91089580E090E008950895E8
:1046900080916A0380FF0BC060912A0185E0689FCA
:1046A000B001112475956795759567952BC081FFAD
:1046B00009C060912A0185E0689FB00111247595B9
:1046C000679520C082FF07C060912A0185E0689F3E
:1046D000B001112417C090916B039923D1F0609120
:1046E0002901961788F720912A0185E0289F9001DB
:1046F0001124929FA001939F500D112470E0CA01D4
:104700000E94F22A6038710540F46115710519F4B0
:1047100006C065E070E0862F08958FE7089581E078
:10472000089580916A0380FF08C06091280170E0BD
:10473000759567957595679521C081FF06C0609155
:10474000280170E07595679519C082FF04C06091DB
:10475000280170E010C090916B03992399F060914B
:1047600027019617A0F780912801899FC001112485
:1047700070E00E94F22A6038710540F461157105FD
:1047800019F406C061E070E0862F08958FE7089560
:1047900081E00895803F21F40E944823819504C060
:1047A000813F29F40E94482380936E030895823F3D
:1047B00021F40E944823819504C0833F29F40E947C
:1047C000482380936D030895893F19F40E94912333
:1047D00005C08A3F31F40E949123819580936F0335
:1047E00008958B3F21F40E949123819504C08C3F52
:1047F00029F40E949123809370030895843F21F44B
:1048000080916C03816017C0853F21F480916C0317
:10481000826011C0863F21F480916C0384600BC0DC
:10482000873F21F480916C03886005C0883F31F494
:1048300080916C03806180936C0308958D3F21F417
:1048400080916A0381600BC08E3F21F480916A03DE
:10485000826005C08F3F29F480916A038460809351
:104860006A030895803F39F480916E0387FF6CC01E
:1048700010926E0369C0813F29F480916E0318166F
:10488000BCF362C090916D03823F29F497FF5CC036
:1048900010926D0359C0833F19F41916CCF354C01C
:1048A000893F41F480916F0318160CF04DC01092AF
:1048B0006F034AC08A3F29F480916F0387FF44C089
:1048C000F6CF8B3F39F48091700387FF3DC0109283
:1048D00070033AC08C3F29F4809170031816BCF322
:1048E00033C0843F21F480916C038E7F17C0853FD5
:1048F00021F480916C038D7F11C0863F21F480915B
:104900006C038B7F0BC0873F21F480916C03877F02
:1049100005C0883F31F480916C038F7E80936C03D7
:1049200013C08D3F21F480916A038E7F0BC08E3FB0
:1049300021F480916A038D7F05C08F3F29F4809117
:104940006A038B7F80936A0380916D0381110EC08F
:1049500080916E0381110AC080916F03811106C09E
:1049600080917003811102C010926B0308958091B1
:10497000620383FF7EC08DE395E00E94E60580918F
:104980006C031F928F9388E395E09F938F930E940F
:104990007F0686E395E00E94E60580916D03282F4F
:1049A000082E000C330B3F938F9383E395E09F9386
:1049B0008F930E947F0681E395E00E94E605809137
:1049C0006E03282F082E000C330B3F938F938EE23B
:1049D00095E09F938F930E947F068CE295E00E9462
:1049E000E60580916F03282F082E000C330B3F93B0
:1049F0008F9389E295E09F938F930E947F0687E2D1
:104A000095E00E94E60580917003282F082E000C87
:104A1000330B3F938F9384E295E09F938F930E9493
:104A20007F0681E295E00E94E60580916B031F926C
:104A30008F938EE195E09F938F930E947F068CE188
:104A400095E00E94E60580916A031F928F9389E1A9
:104A500095E09F938F930E947F0686E195E00E94E8
:104A6000E6058DB79EB74C960FB6F8949EBF0FBE65
:104A70008DBF8CE693E00E9451150E948622909390
:104A800069038093680308951F93CF93DF93809108
:104A90006803909169030E949E22AC0190916B0380
:104AA000992321F020912B0130E006C020912C01A8
:104AB0008AE0289F900111244217530708F485C00B
:104AC00080916D03C0916E03D0916F0310917003BC
:104AD000811107C0C11175C0D11173C0111171C00E
:104AE00074C09F3F19F09F5F90936B03181624F4D6
:104AF0000E94482380936D0380916D0387FF05C05A
:104B00000E944823819580936D031C1624F40E9413
:104B1000482380936E0380916E0387FF05C00E9437
:104B20004823819580936E0360916D03662331F174
:104B3000C0916E03CC2311F1062E000C770B880B6D
:104B4000990B0E94F92923E333E343E35FE30E94D7
:104B50005D2A0E94C12960936D036C2FCC0F770BE7
:104B6000880B990B0E94F92923E333E343E35FE3C6
:104B70000E945D2A0E94C12960936E031D1624F4D1
:104B80000E94912380936F0380916F0387FF05C07C
:104B90000E949123819580936F03111624F40E9443
:104BA0009123809370038091700387FF05C00E945A
:104BB0009123819580937003DF91CF911F910C9485
:104BC000B7249F3F09F08FCFA0CFDF91CF911F91E6
:104BD0000895ECE6F3E085E0DF011D928A95E9F7A0
:104BE00010926B0310926A03089580E697E00E948A
:104BF000E6051F9281E08F931F9285E08F9382E1FB
:104C000097E09F938F930E947F060F900F900F90D5
:104C10000F900F900F9008958330E9F128F48130C0
:104C200061F0823009F10895853009F462C008F41A
:104C300049C0863009F474C0089580912C01262F54
:104C400030E0280F311D2F3F310524F4680F6093A9
:104C50002C0103C08FEF80932C0180912C011F92B7
:104C60008F938BE496E072C080912B01262F30E069
:104C7000280F311D2F3F310524F4680F60932B015D
:104C800003C08FEF80932B0180912B011F928F9394
:104C900089E396E05BC080912A01262F30E0280F3F
:104CA000311D2F3F310524F4680F60932A0103C0A2
:104CB0008FEF80932A0180912A011F928F9386E2C1
:104CC00096E044C080912901262F30E0280F311D45
:104CD0002F3F310524F4680F6093290103C08FEF43
:104CE00080932901809129011F928F9381E196E0A1
:104CF0002DC080912801262F30E0280F311D2F3F35
:104D0000310524F4680F6093280103C08FEF80936E
:104D10002801809128011F928F9388EF95E016C09B
:104D200080912701262F30E0280F311D2F3F3105BC
:104D300024F4680F6093270103C08FEF809327014D
:104D4000809127011F928F938DED95E09F938F9314
:104D50000E947F060F900F900F900F900895833060
:104D600081F128F4813059F08230D1F008958530F6
:104D700009F449C0B8F1863009F456C0089580910D
:104D80002C01681720F4861B80932C0102C010921E
:104D90002C0180912C011F928F938EEC95E054C0D2
:104DA00080912B01681720F4861B80932B0102C091
:104DB00010922B0180912B011F928F938CEB95E029
:104DC00043C080912A01681720F4861B80932A0132
:104DD00002C010922A0180912A011F928F9389EAC2
:104DE00095E032C080912901681720F4861B8093DA
:104DF000290102C010922901809129011F928F93ED
:104E000084E995E021C080912801681720F4861B71
:104E10008093280102C010922801809128011F92DE
:104E20008F938BE795E010C080912701681720F4DD
:104E3000861B8093270102C01092270180912701D1
:104E40001F928F9380E695E09F938F930E947F0639
:104E50000F900F900F900F900895CF93C82F1F922F
:104E60008F9385E698E09F938F930E947F0681E061
:104E700090E0A0E0B0E0BC01CD0104C0660F771F58
:104E8000881F991FCA95D2F70E94B41F0F900F90E8
:104E90000F900F90CF910C943418CF93873288F5F0
:104EA0008E3108F00BC18E3009F487C0D8F48730FA
:104EB00009F460C08B3009F44FC0863009F002C19C
:104EC00080916203817F8E7F809362038AE698E0FF
:104ED0000E94E6058CE19BE00E94E60581E080935C
:104EE000720346C0863109F4B0C020F4803109F461
:104EF0007AC0E8C0893109F491C08B3109F449C006
:104F0000E1C0883349F150F4893209F4D5C08533C2
:104F100009F4D2C0873209F0D5C0CEC0833409F479
:104F2000CBC028F48A3308F4CDC08953C8C0883474
:104F300009F0C8C00E9434188BE09BE00E94E6058F
:104F40002FEF83ED90E3215080409040E1F700C0C7
:104F500000000E94ED220CC081E998E041C082EF80
:104F60009AE00E94E605809162038160809362036B
:104F7000C1E0ADC080916203C82FC17080FFEFCF48
:104F80008EEF9AE00E94E60580916203817F8E7F1A
:104F90003FC09091620391FBCC27C0F981E0C82704
:104FA000892FC0FB81F980936203CC2319F085EE31
:104FB0009AE029C087ED9AE013C09091620392FBBA
:104FC000CC27C0F981E0C827892FC0FB82F98093E4
:104FD0006203CC2319F088EC9AE015C088EB9AE0C4
:104FE0000E94E605C5CF9091620393FBCC27C0F9E0
:104FF00081E0C827892FC0FB83F980936203CC230B
:1050000051F08CEA9AE00E94E6058091620381608B
:10501000809362035CC08FE99AE0E2CF80E99AE076
:105020000E94E6058DE69AE00E94E60588E29AE095
:105030000E94E6058FEF99E00E94E6058AEB99E071
:105040000E94E6058FE899E0CBCF81E899E00E94C5
:10505000E6050E94FC141F928F9387E699E09F93C8
:105060008F930E947F06809124011F928F9380E589
:1050700099E09F938F930E947F0680917F021F92F9
:105080008F938DE399E09F938F930E947F060E94F8
:1050900092229F938F937F936F9386E299E09F93E1
:1050A0008F930E947F068DB79EB742960FB6F894F5
:1050B0009EBF0FBE8DBF5CCF80E001C08D510E94AE
:1050C0002D2756CF84E299E00E94E605C0E08C2FA0
:1050D000CF91089580E008950C946A28CF93C82F4B
:1050E00080917203813069F020F0823009F449C068
:1050F00040C167E08FE00E946716882309F43FC132
:1051000006C067E08FE00E946716882361F08C2F4D
:105110000E946C28811104C08C2F0E944D272FC043
:1051200081E090E02CC08C2F0E946A28811126C05B
:10513000C431E1F070F4CB3081F0C031D1F40E9481
:10514000F5258DE598E00E94E60582E080937203E4
:1051500015C0C93259F0C83361F48AE698E00E945C
:10516000E60581E698E00E94E60508C01092720309
:1051700004C18BE598E00E94E605FFC081E08170E4
:10518000FEC0C43228F5CE3108F0C1C0CB30A1F149
:10519000D0F4C73009F0D3C08EE180932C0182E3B4
:1051A00080932B018AE080932A0184E18093290176
:1051B00088E08093280188E28093270181E097E0CE
:1051C0000E94E605BFC0C33149F1C431C1F0B7C088
:1051D000CB3409F4A9C028F4C93289F0C83361F08E
:1051E000AEC0C13509F49EC0C23509F499C0CE34B1
:1051F00009F0A5C06AE09EC00E94F525A3C0809179
:105200007103882319F0109271039CC08EE097E01F
:105210000E94E60581E080937203B1C088EE96E0BB
:105220000E94E60586ED96E00E94E60580912C013D
:105230001F928F9383ED96E09F938F930E947F063A
:1052400081ED96E00E94E6058FEB96E00E94E60570
:1052500080912B011F928F938CEB96E09F938F93FD
:105260000E947F068AEB96E00E94E6058BEA96E0B4
:105270000E94E60580912A011F928F9388EA96E0AA
:105280009F938F930E947F0686EA96E00E94E60530
:1052900085E996E00E94E605809129011F928F938F
:1052A00082E996E09F938F930E947F0680E996E0C3
:1052B0000E94E6058BE796E00E94E60580912801B2
:1052C0001F928F9388E796E09F938F930E947F06AB
:1052D00086E796E00E94E6058FE596E00E94E605E7
:1052E000809127011F928F938CE596E09F938F9377
:1052F0000E947F068AE596E00E94E6058DB79EB77C
:1053000048960FB6F8949EBF0FBE8DBF1BC0CE51FE
:10531000EC2FF0E0E85BFE4F80818093710312C0B8
:1053200061E003C061E006C06AE0809171030E9401
:105330000C2608C0809171030E94AF2603C08FEF36
:1053400096E013C080917103882369F01F928F93B8
:1053500089EF96E09F938F930E947F060F900F90A6
:105360000F900F9004C086EF96E00E94E60581E062
:1053700006C01092720380E002C080E000CFCF919F
:1053800008950E94C8296894B1110C94572A089571
:105390000E943C2A88F09F5798F0B92F9927B7515F
:1053A000B0F0E1F0660F771F881F991F1AF0BA95C9
:1053B000C9F714C0B13091F00E94562AB1E00895A7
:1053C0000C94562A672F782F8827B85F39F0B93F99
:1053D000CCF3869577956795B395D9F73EF490957C
:1053E0008095709561957F4F8F4F9F4F0895E894FA
:1053F00009C097FB3EF490958095709561957F4F1D
:105400008F4F9F4F9923A9F0F92F96E9BB279395CA
:10541000F695879577956795B795F111F8CFFAF4DA
:10542000BB0F11F460FF1BC06F5F7F4F8F4F9F4F0B
:1054300016C0882311F096E911C0772321F09EE869
:10544000872F762F05C0662371F096E8862F70E0CF
:1054500060E02AF09A95660F771F881FDAF7880FA9
:105460009695879597F9089557FD9058440F551FC5
:1054700059F05F3F71F04795880F97FB991F61F0D6
:105480009F3F79F087950895121613061406551F4D
:10549000F2CF4695F1DF08C0161617061806991FB9
:1054A000F1CF86957105610508940895E894BB27AE
:1054B00066277727CB0197F908950E94702A0C94EC
:1054C000E12A0E94D32A38F00E94DA2A20F095239C
:1054D00011F00C94CA2A0C94D02A11240C94572A47
:1054E0000E94342A70F3959FC1F3950F50E0551F29
:1054F000629FF001729FBB27F00DB11D639FAA2729
:10550000F00DB11DAA1F649F6627B00DA11D661F77
:10551000829F2227B00DA11D621F739FB00DA11D98
:10552000621F839FA00D611D221F749F3327A00D52
:10553000611D231F849F600D211D822F762F6A2FEE
:1055400011249F5750409AF0F1F088234AF0EE0F53
:10555000FF1FBB1F661F771F881F91505040A9F780
:105560009E3F510580F00C94CA2A0C94572A5F3F45
:10557000E4F3983ED4F3869577956795B795F795BC
:10558000E7959F5FC1F7FE2B880F911D9695879534
:1055900097F9089597F99F6780E870E060E00895B3
:1055A0009FEF80EC089500240A941616170618063B
:1055B0000906089500240A94121613061406050617
:1055C0000895092E0394000C11F4882352F0BB0FA8
:1055D00040F4BF2B11F460FF04C06F5F7F4F8F4F0B
:1055E0009F4F089597FB072E16F4009407D077FD80
:1055F00009D00E940C2B07FC05D03EF490958195B4
:105600009F4F0895709561957F4F0895EE0FFF1F8E
:105610000590F491E02D0994AA1BBB1B51E107C032
:10562000AA1FBB1FA617B70710F0A61BB70B881F32
:10563000991F5A95A9F780959095BC01CD010895C1
:04564000F894FFCF0C
:10564400FFFFA514000069FFFF27E78C000000FF9F
:10565400FF9464000576010000FF820C120DEF0C2C
:10566400B90C850C0158032808140A321E79657395
:10567400006E6F00404D36227E043104FB03D903D3
:1056840065037E039703B0030102030405060708BC
:0256940009000B
:106800008800EA44E944E244040005000600070069
:10681000080009000A000B000C000D000E000F001C
:1068200010001100120013001400150016001700CC
:10683000180019001A001B001C001D001E001F007C
:10684000200021002200230024002500260027002C
:10685000280029002A002B002C002D002E002F00DC
:10686000300031A232003300340035A13600370049
:10687000380082003A003B003C003D003E003F00F3
:1068800040004100420043004400450046004700EC
:10689000480049004A004B004C004D004E004F009C
:1068A000500051005200530067005400550056003C
:1068B000580059005A005B005C005D005E005F00FC
:1068C00060006100620063006400650057006700BB
:1068D000CD4469006A006B006C006D006E006F00B3
:1068E0007000710072006620890087008A008B00AA
:1068F000E000E100E200E300E400E500E600E7007C
:106900008800010001000100EA4401000100E244A6
:106910000100010001000100460001004A004B0097
:10692000010001004700480001000100E9440100A6
:106930000100010001000100010001003A003B00DC
:106940003C003D003E003F0040004100420043004B
:10695000010035004C0001000100440045005200D8
:1069600049000100010050004F0029004D004E0079
:1069700051000100010001000100010001000100BF
:1069800001000100010001000100010001000100FF
:1069900001000100010001000100010001004D00A3
:1069A0004A004E004B0001000100010001000100FF
:1069B00001000100010001000100010001000100CF
:1069C00001000100010001000100650001006700F5
:1069D000010069006A006B006C006D006E006F00C2
:1069E0007000710072000100890087008A008B002E
:1069F0000100010001000100010001000100E700A9
:106A00008800010001000100EA4401000100E244A5
:106A10000100010001000100460001004A004B0096
:106A2000010001004700480001000100E9440100A5
:106A30000100010001000100010001003A003B00DB
:106A40003C003D003E003F0040004100420043004A
:106A5000010035004C0001000100440045005200D7
:106A600049000100010050004F0029004D004E0078
:106A700051000100010001000100010001000100BE
:106A800001000100010001000100010001000100FE
:106A900001000100010001000100010001004D00A2
:106AA0004A004E004B0001000100010001000100FE
:106AB00001000100010001000100010001000100CE
:106AC00001000100010001000100650001006700F4
:106AD000010069006A006B006C006D006E006F00C1
:106AE0007000710072000100890087008A008B002D
:106AF0000100010001000100010001000100E700A8
:00000001FF
